S018000064656D6F70726F675F7333326B3134342E7372656374
S11320000070002029250000912500009125000082
S1132010912500009125000091250000000000009A
S113202000000000000000000000000091250000F6
S1132030912500000000000091250000ED2B000018
S113204091250000912500009125000091250000B4
S113205091250000912500009125000091250000A4
S11320609125000091250000912500009125000094
S11320709125000091250000912500009125000084
S11323F09125000091250000EE11AA55FFFFFFFF73
S1132400FFFFFFFFFFFFFFFFFFFFFFFFFE7FFFFF59
S1132410044B05481B1A062B02D9044B03B1184779
S1132420704700BF6B84FF1F6884FF1F000000001B
S113243005490648091A891001EBD171491002D0E7
S1132440034B03B1184770476884FF1F6884FF1F5C
S11324500000000010B5064C237843B9FFF7D8FFFD
S1132460044B13B10448AFF300800123237010BD63
S11324700000002000000000782E000008B5084B82
S11324801BB108490848AFF300800848036813B932
S1132490BDE80840CCE7064B002BF9D09847F7E796
S11324A00000000004000020782E00006484FF1F58
S11324B000000000154B002B08BF134B9D46A3F5ED
S11324C0803A00218B460F461348144A121A00F032
S11324D0A3FC0F4B002B00D098470E4B002B00D0D1
S11324E098470020002104000D000D48002802D068
S11324F00C48AFF3008000F06BFC2000290000F0D2
S1132500CDFA00F051FC00BF00000800007000206C
S11325100000000000000000000000207400002003
S1132520000000000000000072B64FF000014FF000
S113253000024FF000034FF000044FF000054FF08D
S113254000064FF00007B846B946BA46BB46BC463B
S11325500A490B4A521A013A05DD00200423086097
S11325601944043AFBDA0748854607488047074878
S1132570804762B6FFF79EFFFEE700000080FF1F62
S11325800070002000700020FD2B0000D12C000002
S1132590FFF7FEBF38B50C4B1B68002B00DB38BDC2
S11325A0094A136823F00043136000F019FB00F19B
S11325B0FA05054C236813F4801FF0D000F010FBDB
S11325C08542F7D2EBE700BF0040024038B50B4B21
S11325D01A6842F080421A601A6842F080521A6007
S11325E000F0FEFA00F1FA05044C236813F0807F32
S11325F003D100F0F5FA8542F7D238BD004002401D
S113260070B582B000238DF8003001238DF80130BD
S113261002238DF8023004238DF8033008238DF84B
S1132620043010238DF8053020238DF80630402324
S11326308DF80730AA4BD3F8AC2122F08042C3F8BE
S1132640AC21D3F8AC2142F08442C3F8AC21A3F509
S11326508053D3F80422C2F3022222B94FF48072C9
S1132660C3F8042201229F4BD3F8081201F00101A0
S11326709D489E4B002908BF034602A90A4412F84C
S1132680082CB3FBF2F39A4AA2FB0323DB0B0733B8
S1132690C3F3CC0343F0E063964A1361964B536152
S11326A000239361136253624FF470339362936A0D
S11326B043F0880393620123D3624FF44023936170
S11326C0A2F5C042D2F8903043F08043C2F8903073
S11326D0FFF760FFFFF77AFF884B1B68002B11DBC5
S11326E0864A136843F00043136000F079FA00F15E
S11326F0FA05824C236813F4801F03D100F070FAAA
S11327008542F7D27D4A536823F400535360FFF7A0
S113271041FFFFF75BFF00238DF8003001238DF8A4
S1132720013002238DF8023004238DF8033008238E
S11327308DF8043010238DF8053020238DF80630F1
S113274040238DF80730674BD3F80431C3F30223D9
S11327502BB94FF48072634BC3F80421012302AAFE
S1132760134413F8083C4FF4FA50B0FBF3F0002282
S11327701446634E4FF4FA7502E00132122A17D060
S113278016F8223005FB03F3B0FBF3F103FB110150
S11327900029F2D1B0FBF3F39CB2611E89B2FF2988
S11327A0EBD8574B03EB820255789178D07802E04E
S11327B0002001460546514A536823F087031B0451
S11327C01B0C53605668631E46EA036353605468E7
S11327D06B1E03F007032343536054684B1EDB0452
S11327E003F46013234353605468431E1B0403F42F
S11327F0E023234353605068042928BF04214B1E5F
S11328009B0503F4400303435360536843F0800380
S1132810536000231046194603F1200240F82210A9
S11328200133802BF8D100233448194603F508728C
S113283040F822100133202BF8D1304B1A6822F0D3
S11328407F0242F01F021A601A6842F400321A60D2
S11328501A6842F480321A601A6822F000521A6030
S11328606FF02042C3F8A4284FF08062C3F810210F
S1132870244AC3F8142100229A624FF0FF321A63EB
S1132880214A1A621A6822F400021A605A6822F471
S1132890805222F008025A601A6822F080421A60BC
S11328A01A6822F080521A6000F09AF900F1FA05D1
S11328B0124C236813F0807F03D000F091F9854215
S11328C0F7D200F08DF900F1FA050C4C236813F0EF
S11328D0006F03D000F084F98542F7D202B070BDD6
S11328E0005006400040064080841E0000127A001A
S11328F0C5B3A29100B0064000C01FC00040024012
S11329002C2E000000009C1906003B0010B582B07C
S11329103D4B1B78002B3FD13C4B5B6913F4001FEC
S113292008D03A4BDB69DBB2394A1370013BDBB2A6
S11329303F2B26D9374B1B6B13F4007F1FD0354B2D
S1132940D3F81001C0F30340002855D00DF1FF3136
S11329500023314C83F00302D2B2125D01F8012F3F
S11329600133DAB29042F5D82A4B4FF400721A635D
S11329709A682A4B1A609DF80030FF2B2CD002B0C5
S113298010BD00F02DF9264B186001221E4B1A7061
S11329900022244B1A70CDE71C4B5B6913F4001F13
S11329A01FD020490B78194AD469194AD0184470A9
S11329B00133DBB20B7012789A42BBD10022124B66
S11329C01A70134B5B78FF2BB4D1114B9B78002BFF
S11329D0B0D100F071F9ADE70228D0D100F06CF964
S11329E0CDE700F0FDF80E4B1B6864339842A1D983
S11329F00022054B1A709DE7064B4FF400721A63D0
S1132A009A68064B1A60BAE76100002000B00640DD
S1132A102000002000400240184102401C00002019
S1132A206400002062000020074A136843F48073A6
S1132A301360064B5A6942F001025A615A6842F027
S1132A4001025A60704700BF00C00440C0F00F404C
S1132A5008B500F0C5F80E4B1B68C31AB3F5FA7F2E
S1132A600CD30C4B1B7853B901220A4B1A700A4A37
S1132A70936843F001039360054B186008BD00227E
S1132A80044B1A70044A536843F001035360F3E79C
S1132A906C00002068000020C0F00F4008B5414BD6
S1132AA040F20112C3F804212422C3F80821D3F808
S1132AB0002112F4000FFAD101223A4BC3F800218D
S1132AC0D3F8002112F0807FFAD0364BD3F80026D9
S1132AD012F4000FFAD1334BD3F8002622F001028E
S1132AE0C3F80026D3F8042642F4407242F00202EE
S1132AF0C3F804264FF4C012C3F80826D3F80026FE
S1132B0012F4000FFAD1274AD2F8003643F0010339
S1132B10C2F800361346D3F8002612F0807FFAD0AC
S1132B20204B40F20112C3F804221F4A5A611A468C
S1132B301369C3F30363062BFAD100F07DF81B4B32
S1132B40D3F82C2142F08042C3F82C21D3F8302151
S1132B5042F08042C3F83021D3F8342142F080425D
S1132B60C3F83421A3F5D0339A6942F400729A6110
S1132B70DA6942F40072DA6103F500531A6942F427
S1132B80A0621A615A6942F4A0625A6100F010F816
S1132B90FFF74AFF62B6FFF733FDFFF759FFFFF770
S1132BA0B5FEFAE700400640120001060050064058
S1132BB0074B1B68074AA2FB03239B09013B064AF8
S1132BC053600023936007211160044A1360704727
S1132BD00084FF1FD34D621010E000E0700000205D
S1132BE0014B1868704700BF70000020024A136848
S1132BF001331360704700BF700000204FF0E023E2
S1132C00D3F8882D42F47002C3F8882DD3F8342FFA
S1132C1022F08042C3F8342F054B064A5A605A68A2
S1132C2042F220121A604FF6FF729A60704700BF9A
S1132C300020054020C528D91B4B1A691B69C3F322
S1132C400363013B052B2ED8DFE803F025030D2D8C
S1132C502D12154BD3F8083203F00103002B13494E
S1132C6018BF0B4618E0104BD3F80833104B13E091
S1132C700D4BD3F80816D3F80836C3F3044303F115
S1132C8010000A4B03FB00F3C1F302210131490098
S1132C90B3FBF1F300E0054BC2F303420132B3FB93
S1132CA0F2F3044A136070470040064000127A00B1
S1132CB0006CDC020084FF1F4FF0E021D1F80C2DE2
S1132CC092B2024B1343C1F80C3D70470400FA055D
S1132CD0264B274A9A4208D013462448254A13F81B
S1132CE0011B02F8011B9842F9D1234B234A9A4253
S1132CF008D013462048224A13F8011B02F8011B8E
S1132D008342F9D11F4B204A9A4206D01346002130
S1132D101C4A03F8011B9342FBD11C4B1C4A9A42E8
S1132D2008D0134619481B4A13F8011B02F8011B6B
S1132D308342F9D1184B194A9A4212D010B4184C54
S1132D40A40808D01946002351F8040B42F8040BD8
S1132D500133A342F8D1134B104A1A605DF8044BB7
S1132D607047104B0C4A1A60704700BF082F0000D0
S1132D70A02E00000084FF1F082F0000082F000071
S1132D806884FF1F7400002000000020082F00004A
S1132D90082F000000000020002000000080FF1F1A
S1132DA00004000008ED00E008B5074B044613B129
S1132DB00021AFF30080054B1868836A03B198477C
S1132DC0204600F031F800BF00000000742E00001F
S1132DD070B50D4E0D4CA41BA4100025A54209D1BD
S1132DE00B4E0C4C00F048F8A41BA4100025A5427F
S1132DF005D170BD56F8253098470135EEE756F8F1
S1132E00253098470135F2E7982E0000982E0000EF
S1132E10982E00009C2E000002440346934200D1E9
S1132E20704703F8011BF9E7FEE7000008030202FC
S1132E30090303020A0303030B0403030C0404033E
S1132E400D0504030E0504040F060404100605040E
S1132E5011070504120705051308050514080605DE
S1132E6015080705160807061708080618080807AE
S1132E70190808080484FF1FF8B500BFF8BC08BC93
S1132E809E467047F8B500BFF8BC08BC9E46704724
S10B2E9024F6FF7F010000009D
S1072E987D24000091
S1072E9C55240000B5
S1132EA0006CDC02000000000000000000000000D4
S1132EB0000000000000000000000000000000000E
S1132EC000000000000000000000000000000000FE
S1132ED000000000000000000000000000000000EE
S1132EE000000000000000000000000000000000DE
S1132EF000000000000000000000000000000000CE
S10B2F000000000000000000C5
S9032529AE
